:100000000C94BA000C947C060C94A1060C94E200AB
:100010000C94E2000C94E2000C94E2000C94E200D8
:100020000C94E2000C94E2000C94E2000C94E200C8
:100030000C94E2000C94E2000C94E2000C94E200B8
:100040000C94B9040C94E2000C9487040C946104A1
:100050000C94E2000C94E2000C94E2000C94E20098
:100060000C94E2000C94E200BC0CBA0CC10CD80C4D
:10007000720DFA0C1B0D370D530D840D820D890D79
:10008000A00DA00DC20DE30DFF0D1B0E91079A07E9
:10009000A507C407EB07F4077B087B087B087B08F0
:1000A0007B087B087B087B08FE0711087B087B0820
:1000B0007B087B08400848084B085708710808006F
:1000C0000000BE922449123EABAAAA2ABECDCCCCD7
:1000D0004C3E00000080BEABAAAAAA3E0000000071
:1000E000BF000000803F0000000000084178D3BB43
:1000F0004387D1133D190E3CC3BD4282AD2B3E68F0
:10010000EC8276BED98FE1A93E4C80EFFFBE01C4E0
:10011000FF7F3F00000000000000000024002700D7
:100120002A0000000000250028002B00000000002D
:100130002300260029000404040404040404020229
:100140000202020203030303030301020408102056
:100150004080010204081020010204081020000061
:100160000008000201000003040700000000000076
:1001700000007C0811241FBECFEFD8E0DEBFCDBF4A
:1001800011E0A0E0B1E0EAE0F5E202C005900D92D6
:10019000A432B107D9F722E0A4E2B1E001C01D9278
:1001A000A034B207E1F710E0CAEBD0E004C0219719
:1001B000FE010E947812C93BD107C9F70E94A90825
:1001C0000C9483120C940000CF92DF92EF92FF9276
:1001D0000F931F93CF93DF936C017A018B01C0E0E3
:1001E000D0E0CE15DF0589F0D8016D918D01D601E3
:1001F000ED91FC910190F081E02DC6010995892BCC
:1002000011F47E0102C02196ECCFC701DF91CF919E
:100210001F910F91FF90EF90DF90CF900895089578
:1002200080E090E00895FC01538D448D252F30E04F
:10023000842F90E0821B930B541710F0CF960895F3
:1002400001970895FC01918D828D981761F0828D40
:10025000DF01A80FB11D5D968C91928D9F5F9F73FA
:10026000928F90E008958FEF9FEF0895FC01918D9C
:10027000828D981731F0828DE80FF11D858D90E009
:1002800008958FEF9FEF0895FC01918D228D892FA6
:1002900090E0805C9F4F821B91098F73992708958E
:1002A0008DE991E00E94440121E0892B09F420E0CE
:1002B000822F0895FC01848DDF01A80FB11DA35A80
:1002C000BF4F2C91848D90E001968F739927848F76
:1002D000A689B7892C93A089B1898C9180648C936D
:1002E000938D848D981306C00288F389E02D808158
:1002F0008F7D80830895EF92FF920F931F93CF938A
:10030000DF93EC0181E0888F9B8D8C8D981305C065
:10031000E889F989808185FD24C0F62E0B8D10E0D7
:100320000F5F1F4F0F731127E02E8C8DE8120CC04A
:100330000FB607FCFACFE889F989808185FFF5CFF0
:10034000CE010E945A01F1CF8B8DFE01E80FF11D05
:10035000E35AFF4FF0820B8FEA89FB89808180622C
:1003600007C0EE89FF896083E889F989808180640C
:10037000808381E090E0DF91CF911F910F91FF90FA
:10038000EF900895CF93DF93EC01888D8823C9F017
:10039000EA89FB89808185FD05C0A889B9898C918E
:1003A00086FD0FC00FB607FCF5CF808185FFF2CF29
:1003B000A889B9898C9185FFEDCFCE010E945A01A1
:1003C000E7CFDF91CF91089580E090E0892B29F06D
:1003D0000E94500181110C9400000895833081F037
:1003E00028F4813099F08230A1F008958730A9F087
:1003F0008830B9F08430D1F4809180008F7D03C0C3
:10040000809180008F7780938000089584B58F77E6
:1004100002C084B58F7D84BD08958091B0008F7730
:1004200003C08091B0008F7D8093B0000895CF937A
:10043000DF93282F30E0F901E25AFE4F8491F90151
:10044000E65BFE4FD491F901EA5CFE4FC491CC23E8
:1004500091F081110E94EE01EC2FF0E0EE0FFF1FF2
:10046000E45DFE4FA591B491EC91ED2381E090E025
:1004700021F480E002C080E090E0DF91CF91089508
:100480001F93CF93DF93282F30E0F901E25AFE4FFC
:100490008491F901E65BFE4FD491F901EA5CFE4FCD
:1004A000C491CC23C9F0162F81110E94EE01EC2FCC
:1004B000F0E0EE0FFF1FEE5DFE4FA591B4918FB7F8
:1004C000F894111105C09C91ED2FE095E92302C02D
:1004D000EC91ED2BEC938FBFDF91CF911F9108959D
:1004E000CF93DF9390E0FC01E65BFE4F2491FC018B
:1004F000EA5CFE4F8491882361F190E0880F991F98
:10050000FC01E85EFE4FC591D491FC01EE5DFE4F0B
:10051000A591B491611109C09FB7F8948881209585
:1005200082238883EC912E230BC0623061F49FB745
:10053000F8943881822F809583238883EC912E2B29
:100540002C939FBF06C08FB7F894E8812E2B288389
:100550008FBFDF91CF9108958E3008F08E50877055
:10056000806480937C0080917A00806480937A001C
:1005700080917A0086FDFCCF8091780020917900EF
:1005800090E0922B08953FB7F894809139019091B3
:100590003A01A0913B01B0913C0126B5A89B05C052
:1005A0002F3F19F00196A11DB11D3FBFBA2FA92FF2
:1005B000982F8827820F911DA11DB11DBC01CD016F
:1005C00042E0660F771F881F991F4A95D1F708955B
:1005D0008F929F92AF92BF92CF92DF92EF92FF9253
:1005E0006B017C010E94C3024B015C01C114D10468
:1005F000E104F104F1F00E94C302DC01CB0188198F
:100600009909AA09BB09883E9340A105B10570F379
:1006100021E0C21AD108E108F10888EE880E83E0D3
:10062000981EA11CB11CC114D104E104F10419F7F6
:10063000DDCFFF90EF90DF90CF90BF90AF909F9075
:100640008F9008952FB7F89460913501709136011D
:1006500080913701909138012FBF08958F929F921A
:10066000AF92BF92CF92DF92EF92FF9284E10E940D
:10067000AC02BC01990F880B990B0E94D11020E0AD
:1006800030E040E85AE30E94D61120E030E040EA32
:1006900050E40E94D6116B017C01809100018823F7
:1006A00051F0C0923001D0923101E0923201F092CB
:1006B00033011092000126E636E646E65FE36091DC
:1006C00030017091310180913201909133010E948B
:1006D000D6114B015C0120ED3CEC4CEC5DE3C70115
:1006E000B6010E94D6119B01AC01C501B4010E9464
:1006F000BD0F60933001709331018093320190936C
:1007000033012DE33CE248E450E40E94D61120E09E
:1007100030E0A9010E94BD0FFF90EF90DF90CF90D5
:10072000BF90AF909F908F90089585E00E94170230
:1007300061E0892B09F060E085E00E94400287E0DB
:100740000E94170261E0892B09F060E087E00E94B7
:10075000400284E00E94170261E0892B09F060E00A
:1007600084E00E94400280E10E94170261E0892B30
:1007700009F060E080E10C9440028DE00E941702D5
:1007800061E0892B09F060E08DE00C94400281E18A
:100790000E94170261E0892B09F060E081E10C946E
:1007A0004002CF92DF92EF92FF92CF93DF93EC0162
:1007B0000E9422036B017C018B819C81AD81BE81F3
:1007C000B701A601481B590B6A0B7B0B8F819885DB
:1007D000A0E0B0E084179507A607B70708F58A815F
:1007E00080FD02C061E001C060E088810E9440029B
:1007F00088EC90E098878F83CB82DC82ED82FE824A
:100800008A818F5F8A83298190E030E0220F331F35
:100810008217930729F488EE93E098878F831A82D2
:10082000DF91CF91FF90EF90DF90CF9008950E94DD
:100830007E128FE00E94AC02BC01990F880B990BCD
:100840000E94D1109B01AC0160E070EC8FE794E452
:100850000E942E1020E030E040E85FE30E94BC0FD1
:100860009B01AC0160E070E48CE196E40E942E10E4
:1008700020E030E44CE156E40E942E100E948E11DC
:1008800020E030EF47E555E40E942E102FE03FECCA
:100890004BE55BE30E94BD0F9B01AC0160E070E0A3
:1008A00080E89FE30E942E1023E333E948E853E4F5
:1008B0000E94BC0F0E94A01070938A01609389016E
:1008C00008951F920F920FB60F9211242F933F930A
:1008D0004F935F936F937F938F939F93AF93BF9348
:1008E000EF93FF938DE991E00E945A01FF91EF9100
:1008F000BF91AF919F918F917F916F915F914F9138
:100900003F912F910F900FBE0F901F9018951F923F
:100910000F920FB60F9211242F938F939F93EF9303
:10092000FF93E091AD01F091AE018081E091B301C0
:10093000F091B40182FD12C090818091B6018F5F69
:100940008F732091B701821751F0E091B601F0E06A
:10095000E356FE4F958F8093B60101C08081FF91D1
:10096000EF919F918F912F910F900FBE0F901F903D
:1009700018951F920F920FB60F9211242F933F9349
:100980008F939F93AF93BF938091350190913601E0
:10099000A0913701B09138013091340123E0230F49
:1009A0002D3720F40196A11DB11D05C026E8230FA7
:1009B0000296A11DB11D20933401809335019093BF
:1009C0003601A0933701B09338018091390190919D
:1009D0003A01A0913B01B0913C010196A11DB11DCE
:1009E0008093390190933A01A0933B01B0933C016D
:1009F000BF91AF919F918F913F912F910F900FBE1B
:100A00000F901F90189561E084E00E94400261E021
:100A100080E10C9440021092920110929101109288
:100A20008900109288008091950181110C94030532
:100A3000089561E085E00E94400261E087E00C9447
:100A40004002109294011092930110928B00109228
:100A50008A008091950181110C9419050895CF9316
:100A6000DF93EB011C161D0684F4813031F461E044
:100A700085E00E94400260E011C08230E1F561E053
:100A800084E00E94400260E014C02097B1F0813001
:100A900049F460E085E00E94400261E087E00E9446
:100AA00040021BC0823039F560E084E00E944002C1
:100AB00061E080E10E94400220C09091950199235D
:100AC00051F0813019F40E94190507C0823011F5E8
:100AD0000E94030512C0813071F4D0939401C09339
:100AE0009301D7FF03C0D195C195D109D0938B0055
:100AF000C0938A000FC0823069F4D0939201C093F2
:100B00009101D7FF03C0D195C195D109D093890038
:100B1000C0938800DF91CF910895CF92DF92EF923A
:100B2000FF920F931F93CF93C82F0E94C302C1114E
:100B300014C04B9B09C060932801709329018093D6
:100B40002A0190932B01D0C0009128011091290116
:100B500020912A0130912B0116C0C13009F0C4C088
:100B60004A9B09C060932C0170932D0180932E0144
:100B700090932F01B9C000912C0110912D0120916B
:100B80002E0130912F016B017C01C01AD10AE20ABB
:100B9000F30A970186014C2F50E0E0E2CE1AE3E021
:100BA000DE0AE108F108E9E7CE16E5E0DE06E10439
:100BB000F10408F069C0FA01EE0FFF1FEE0FFF1FEE
:100BC000EB59FE4F6083718382839383FA01EA5D60
:100BD000FE4F80818130B1F0823019F0811175C0F3
:100BE00005C01082FA01EC5DFE4F09C0DA01AC5D70
:100BF000BE4F8C918F5F8C93853008F466C081E086
:100C0000808363C0CF5FD901C801875D9540A1098A
:100C1000B1090B97A105B10558F4C13019F40E9430
:100C2000210553C0C23009F050C00E940B054DC0D1
:100C3000083E83E018072105310538F0013DE7E063
:100C40001E0728F000ED17E002C008EE13E0C8010F
:100C5000A0E0B0E09C01AD01285E3340410951099C
:100C6000AAEFB2E00E94800F28EE33E040E050E0AF
:100C70000E94610FCA01B9016D5771408109910944
:100C80008C2F0E942F0521C0FA01EE0FFF1FEE0FDF
:100C9000FF1FEB59FE4F0081118122813381DC015E
:100CA000CB01801B910BA20BB30B813A9648A1405C
:100CB000B10558F0FA01EA5DFE4F82E08083FA0147
:100CC000EC5DFE4F1082CF5FA8CF809126019091FE
:100CD0002701891739F0813011F0913011F481E04A
:100CE00001C082E080937101CF911F910F91FF901D
:100CF000EF90DF90CF9008951F920F920FB60F9252
:100D000011242F933F934F935F936F937F938F9310
:100D10009F93AF93BF93EF93FF9381E00E948D0564
:100D2000FF91EF91BF91AF919F918F917F916F91C3
:100D30005F914F913F912F910F900FBE0F901F9099
:100D400018951F920F920FB60F9211242F933F9375
:100D50004F935F936F937F938F939F93AF93BF93C3
:100D6000EF93FF9380E00E948D05FF91EF91BF917B
:100D7000AF919F918F917F916F915F914F913F9133
:100D80002F910F900FBE0F901F901895CF92DF926A
:100D9000EF92FF926B017C01E091AD01F091AE0109
:100DA00082E08083C11481EED806E104F104B1F041
:100DB00060E079E08DE390E0A70196010E948B0F3F
:100DC000DA01C9010197A109B109B695A7959795CF
:100DD00087959C01211580E13807B8F0E091AD01BD
:100DE000F091AE01108260E874E88EE190E0A70116
:100DF00096010E948B0FDA01C9010197A109B1097F
:100E0000B695A795979587959C01E091A901F091DA
:100E1000AA013083E091AB01F091AC0120831092E4
:100E2000B501E091B101F091B20186E08083E091DB
:100E3000AF01F091B001808180618083E091AF01CA
:100E4000F091B001808188608083E091AF01F091E2
:100E5000B001808180688083E091AF01F091B001A2
:100E600080818F7D8083FF90EF90DF90CF900895F9
:100E7000CF93C1E08DE991E00E944401892BF9F004
:100E80008DE991E00E94220190919C01981307C086
:100E9000C0933F0290933B02C0933A02EBCF9091F4
:100EA0003F02992339F3E0913A0291E09E0F90932B
:100EB0003A02F0E0E55CFD4F80839430D8F28091F7
:100EC0003A02843010F480E01DC090913B02909370
:100ED000980130913C023093990180913D028093BA
:100EE0009A0120913E0220939B01930F890F982F26
:100EF0009F7781E0921380E010923B0210923F02B4
:100F000010923A02CF910895E09199018E2F90E0CE
:100F10008931910508F0EFC0FC01EA5BFF4F0C94AA
:100F2000781260919A0167FD6FE723E0629FB0013C
:100F3000112408C060919A0167FD6FE74DEF4603E9
:100F4000B001112481E00C942F0560919A01633364
:100F500008F0D1C070E080E090E00E94CF102DEC4E
:100F60003CEC4CE45EE30E94D61120E030E040EC23
:100F700050E40E94BD0F60930E0170930F018093A7
:100F8000100190931101089560919A0182EE860FED
:100F90008F3608F0B0C080910D01262F30E045E07B
:100FA000849FC0011124821793070CF4A4C070E041
:100FB00080E090E00E94CF102DEC3CEC4CE45EE32E
:100FC0000E94D6116093090170930A0180930B016E
:100FD00090930C01089560919A0167FD6FE783E09B
:100FE000689FB001112408C060919A0167FD6FE706
:100FF0002DEF2603B001112482E0A5CF80919A0144
:10100000811103C010929701089544E6849FC001A6
:101010001124909308018093070181E08093970148
:10102000089580919A018330B9F028F4813049F015
:10103000823061F008958530C9F098F08630D9F09B
:10104000089560E679E080E090E004C060E875E231
:1010500080E090E00C94C60660E07BE480E090E0E5
:10106000F9CF60E076E980E090E0F4CF60E072ECE8
:1010700081E090E0EFCF60E071EE80E090E0EACFB9
:1010800080919A018093B30081E080939601089546
:1010900010929601089580919A019FEF980F9E31CA
:1010A00050F590E09093060180930501089580919A
:1010B0009A01882399F081E08093950180919301B2
:1010C00090919401892B11F40E941905809191014E
:1010D00090919201892B79F40C940305109295015B
:1010E000089580919A01882321F081E080939001F6
:1010F0000895109290010895EDE9F1E013821282B3
:1011000088EE93E0A0E0B0E084839583A683B78364
:1011100086E191E09183808385EC90E095878487D8
:1011200084EC90E09787868780EC90E0918B808BB1
:1011300081EC90E0938B828B82EC90E0958B848B9A
:1011400086EC90E0978B868B118E128E138E148E08
:101150000895CF93DF9300D000D0CDB7DEB7789459
:1011600084B5826084BD84B5816084BD85B58260AC
:1011700085BD85B5816085BD80916E00816080935D
:101180006E001092810080918100826080938100C6
:1011900080918100816080938100809180008160D6
:1011A000809380008091B10084608093B100809131
:1011B000B00081608093B00080917A008460809359
:1011C0007A0080917A00826080937A0080917A0020
:1011D000816080937A0080917A00806880937A00A1
:1011E0001092C1008EE190E090930401809303017E
:1011F00080E180930D0161E085E00E94700261E072
:1012000087E00E94700261E08AE00E94700260E064
:101210008EE00E94700262E088E00E94700261E04D
:1012200084E00E94700261E080E10E94700261E04F
:1012300089E00E94700260E082E10E94700262E038
:1012400083E10E94700262E08CE00E94700261E023
:101250008BE00E94700260E08FE00E94700262E00A
:1012600083E00E94700262E082E00E94700261E00E
:1012700081E10E94700260E081E10E94400261E031
:101280008DE00E94700260E08DE00E94400281E1EA
:10129000809357018DE08093490162E086E00E94CF
:1012A000700286E00E941702892B11F083E801C0CA
:1012B00084E880939C0160E076E980E090E00E9401
:1012C000C6061092760110928F0182EA8093800008
:1012D00081E18093810087E286BB10926F008DE7E9
:1012E00091E0909387008093860010928500109281
:1012F0008400109289001092880010928B00109246
:101300008A0083E88093B00082E08093B10087E098
:1013100087BB109270001092B2001092B30085E06B
:101320008093690083E08DBB8CBB34E0332E43E0B7
:10133000242E58EC452E512C10918F01111145C1CE
:101340008CE00E941702892B21F425E0C22EC09266
:101350008F010E94220300918B0110918C0120913A
:101360008D0130918E01DC01CB01801B910BA20B12
:10137000B30B893C9105A105B105A8F00E941904A1
:101380000E94220360938B0170938C0180938D01E6
:1013900090938E018091890190918A0187399105FE
:1013A00010F030928F0188E00E941702892B09F417
:1013B000FBC483E10E941702892B09F4F5C40E9443
:1013C00022030091850110918601209187013091BF
:1013D0008801DC01CB01801B910BA20BB30B85367E
:1013E0009105A105B10508F4D9C00E9422034B0163
:1013F0005C016093850170938601809387019093CF
:1014000088018EE00E94AC0260900301709004019C
:10141000869D8001879D100D969D100D1124809151
:101420000201882331F0109344010093430110928C
:101430000201609143017091440180E090E00E94BC
:10144000CF1026E636E646E65FE30E94D6116B0132
:101450007C01B80180E090E00E94CF1020ED3CECD0
:101460004CEC5DE30E94D6119B01AC01C701B601B3
:101470000E94BD0F0E94A0106B017C01709344017B
:1014800060934301209105013091060148EE53E03D
:10149000249FC001259F900D349F900D11248C1521
:1014A0009D0530F4809140018F5F8093400102C020
:1014B0001092400182E10E94AC02869D8001879DCE
:1014C000100D969D100D112480910101882331F09B
:1014D000109342010093410110920101609141017A
:1014E0007091420180E090E00E94CF1026E636E63F
:1014F00046E65FE30E94D61169837A838B839C83DF
:10150000B80180E090E00E94CF1020ED3CEC4CEC64
:101510005DE30E94D6119B01AC0169817A818B81C8
:101520009C810E94BD0F0E94A010709342016093A5
:1015300041012091050130910601E8EEF3E02E9F74
:10154000A0012F9F500D3E9F500D112446175707A5
:1015500030F420913F012F5F20933F0102C0109291
:101560003F01C60ED71ED0923E01C0923D01809130
:1015700040018B3020F480913F018B3078F0109245
:101580003F01109240018092810190928201A092CD
:101590008301B0928401F1E0F0938F010E94220355
:1015A00000917D0110917E0120917F013091800199
:1015B000DC01CB01801B910BA20BB30B853F91404B
:1015C000A105B10508F0F3C3D1C00E9421050E9416
:1015D0000B05133009F494C03CF4113009F472C0C7
:1015E000123009F4A4C0C2C0143021F0153009F43F
:1015F000B4C0BCC00E9422030091790110917A010D
:1016000020917B0130917C01DC01CB01801B910B8F
:10161000A20BB30B89389341A105B105F0F00E94EC
:1016200021050E940B050E94950368EC70E080E0A4
:1016300090E00E94E8020E94950362E370E080E07F
:1016400090E00E94E8020E94220360937901709367
:101650007A0180937B0190937C010E942203009188
:101660008B0110918C0120918D0130918E01DC0154
:10167000CB01801B910BA20BB30B893C9105A105FB
:10168000B10560F00E9419040E94220360938B014F
:1016900070938C0180938D0190938E0188E00E945D
:1016A0001702019709F0B5C383E10E941702019761
:1016B00009F0AFC38091890190918A018639910523
:1016C000B0F0A7C30E942203009181011091820112
:1016D0002091830130918401DC01CB01801B910BAF
:1016E000A20BB30B89389341A105B10518F01092F4
:1016F0008F013CC010927801F6E0F093770136C07C
:101700000E942E0320910E0130910F014091100193
:10171000509111010E94811118160CF07EC30E9495
:101720002203693873418105910508F776C30E9449
:101730002E032091090130910A0140910B01509133
:101740000C010E94291087FF6EC30E942203693892
:1017500073418105910558F666C38CE00E9417021B
:10176000892B29F6309277011092780180918F01B0
:101770008111F0C01092770180917601813009F4D7
:1017800056C0823019F08111E5C0B9C00E943807F7
:10179000882361F00E9484070E94220360937201F3
:1017A00070937301809374019093750180919701F8
:1017B000882321F10E94220300917201109173018C
:1017C0002091740130917501AB01BC01401B510B9C
:1017D000620B730B8091070190910801A0E0B0E0CB
:1017E00084179507A607B70728F40E9421050E94D1
:1017F0000B0582C051E050937801ACC00E942203D7
:101800000091720110917301209174013091750162
:10181000DC01CB01801B910BA20BB30B893E9340E3
:10182000A105B10538F3F2E0F093780193C08091FF
:101830007101813051F0823009F45EC081118AC09B
:1018400092E0C92EC092780185C0809378010E94F1
:10185000220300916D0110916E0120916F01309172
:101860007001DC01CB01801B910BA20BB30B853601
:101870009105A105B10508F46DC00E942203609393
:101880006D0170936E0180936F0190937001F894D5
:101890000E94C302009165011091660120916701C9
:1018A000309168016B017C01C01AD10AE20AF30A87
:1018B00041EAC41646E8D40641E0E406F104D0F05B
:1018C0000091690110916A0120916B0130916C01C6
:1018D000DC01CB01801B910BA20BB30B813A964824
:1018E000A140B10538F00E9421050E940B0582E05D
:1018F0008093710178942EC0209278012BC0809142
:101900007101813029F4809376018093780117C0AA
:101910000E943807882399F0E2E0E09376011DBA2F
:101920000E9484070E9422036093720170937301E6
:101930008093740190937501F1E0F09378018091A8
:101940007601811105C082E0C82EC092770102C0E5
:1019500010927701E09178018E2FEE0F990BAA0B70
:10196000BB0B8930910508F0BDC0FC01EC5CFF4F5A
:101970000C94781261E001C060E081E10E944002B5
:10198000B1C00E9422030091610110916201209177
:10199000630130916401DC01CB01801B910BA20B30
:1019A000B30B8F3E9240A105B10508F49BC015C052
:1019B0000E94220300916101109162012091630154
:1019C00030916401DC01CB01801B910BA20BB30BA6
:1019D0008997A105B10508F485C00E94C7030E943C
:1019E000220360936101709362018093630190937D
:1019F000640178C080916001882321F080915801B2
:101A00008230A1F042E040935801109259011092A7
:101A10005A0110925B0110925C0110925D0150928C
:101A20005F0140925E0151E05093600187E591E0D3
:101A30000E94D10357C080916001882321F08091DA
:101A40005801833099F32092580110925901109255
:101A50005A0110925B0110925C0110925D0150924C
:101A60005F0140925E0181E080936001DFCF809151
:101A70006001882321F0809158018430B9F23092BE
:101A800058011092590110925A0110925B01109264
:101A90005C0110925D0150925F0140925E01E1E0B5
:101AA000E0936001C3CF80916001882329F0809189
:101AB0005801853009F4BACFF5E0F093580110923F
:101AC000590110925A0110925B0110925C01109220
:101AD0005D0150925F0140925E01CC24C394C0929C
:101AE0006001A4CFE09177018E2FEE0F990BAA0B26
:101AF000BB0B8930910508F0BDC0FC01E35CFF4FD2
:101B00000C94781261E001C060E08DE00E94400218
:101B1000B1C00E9422030091530110915401209101
:101B2000550130915601DC01CB01801B910BA20BBA
:101B3000B30B8F3E9240A105B10508F49BC015C0C0
:101B40000E942203009153011091540120915501EC
:101B500030915601DC01CB01801B910BA20BB30B22
:101B60008997A105B10508F485C00E94BD030E94B4
:101B70002203609353017093540180935501909315
:101B8000560178C080915201882321F080914A014A
:101B90008230A1F042E040934A0110924B01109232
:101BA0004C0110924D0110924E0110924F01509233
:101BB00051014092500151E05093520189E491E06B
:101BC0000E94D10357C080915201882321F0809157
:101BD0004A01833099F320924A0110924B011092EE
:101BE0004C0110924D0110924E0110924F015092F3
:101BF00051014092500181E080935201DFCF8091EA
:101C00005201882321F080914A018430B9F2309248
:101C10004A0110924B0110924C0110924D0110920A
:101C20004E0110924F015092510140925001E1E05B
:101C3000E0935201C3CF80915201882329F0809113
:101C40004A01853009F4BACFF5E0F0934A011092C9
:101C50004B0110924C0110924D0110924E011092C6
:101C60004F015092510140925001CC24C394C09234
:101C70005201A4CF8091960181115FC080918F01A4
:101C8000843011F0813029F4DD24DA94D092B3004D
:101C900054C02091890130918A0128323105C8F061
:101CA00027343105C0F4C901A0E0B0E09C01AD01CA
:101CB0002852310941095109AFEAB0E00E94800F72
:101CC0002EE130E040E050E00E94610F10E5120F7D
:101CD00003C010E001C01FEF8091430190914401C7
:101CE00020914101309142012817390708F49C01E5
:101CF000203747E13407C8F0213E5EE23507D0F4D3
:101D0000C901A0E0B0E09C01AD0120573741410975
:101D10005109AFEAB0E00E94800F20E737E140E0D0
:101D200050E00E94610F205B01C020E0211718F4F1
:101D3000212F01C02FEF2093B300809190018823C1
:101D400081F10E94220300914501109146012091EA
:101D5000470130914801DC01CB01801B910BA20BA4
:101D6000B30B0D97A105B105E0F08091930190911F
:101D70009401009709F05DC00E94190580919101BE
:101D800090919201009709F078C00E9403050E948B
:101D9000220360934501709346018093470190931D
:101DA00048010E94E401C8CA30928F0108CB0E940A
:101DB0002E036B017C010E94220360937D017093CE
:101DC0007E0180937F019093800120910E013091DC
:101DD0000F014091100150911101C701B6010E94FD
:101DE000291087FF03C020928F01C0CC20910901E8
:101DF00030910A0140910B0150910C01C701B601CD
:101E00000E94811118160CF0B1CC42E040938F0172
:101E1000ADCC1092780185E009C010927801E7E01E
:101E2000E0937701A3CC1092780188E0809377014A
:101E30009DCC97FF03C091958195910920919101C7
:101E40003091920137FF03C031952195310925501A
:101E50003109821793070CF091CF0E94190563E0B6
:101E600070E080E090E00E94E80260919301709140
:101E7000940181E00E942F0581CF97FF03C09195C7
:101E800081959109209193013091940137FF03C00E
:101E900031952195310925503109821793070CF0AE
:101EA00076CF0E94030563E070E080E090E00E943E
:101EB000E802609191017091920182E00E942F05E9
:101EC00066CF052E97FB1EF400940E94780F57FDF5
:101ED00007D00E948B0F07FC03D04EF40C94780FB0
:101EE00050954095309521953F4F4F4F5F4F089546
:101EF00090958095709561957F4F8F4F9F4F089576
:101F00000E94AD0FA59F900DB49F900DA49F800DD2
:101F1000911D11240895A1E21A2EAA1BBB1BFD01DD
:101F20000DC0AA1FBB1FEE1FFF1FA217B307E407B8
:101F3000F50720F0A21BB30BE40BF50B661F771F10
:101F4000881F991F1A9469F76095709580959095F0
:101F50009B01AC01BD01CF010895A29FB001B39FC9
:101F6000C001A39F700D811D1124911DB29F700DA2
:101F7000811D1124911D08955058BB27AA270E9446
:101F8000D40F0C9447110E94391138F00E9440116F
:101F900020F039F49F3F19F426F40C9436110EF416
:101FA000E095E7FB0C943011E92F0E94581158F38B
:101FB000BA17620773078407950720F079F4A6F52E
:101FC0000C947A110EF4E0950B2EBA2FA02D0B0174
:101FD000B90190010C01CA01A0011124FF27591B6E
:101FE00099F0593F50F4503E68F11A16F040A22F74
:101FF000232F342F4427585FF3CF469537952795E5
:10200000A795F0405395C9F77EF41F16BA0B620BE3
:10201000730B840BBAF09150A1F0FF0FBB1F661F2A
:10202000771F881FC2F70EC0BA0F621F731F841F6D
:1020300048F4879577956795B795F7959E3F08F093
:10204000B0CF9395880F08F09927EE0F9795879555
:1020500008950E940C1108F481E008950E94421036
:102060000C9447110E94401158F00E94391140F021
:1020700029F45F3F29F00C94301151110C947B111D
:102080000C9436110E94581168F39923B1F355232B
:1020900091F3951B550BBB27AA276217730784077B
:1020A00038F09F5F5F4F220F331F441FAA1FA9F311
:1020B00035D00E2E3AF0E0E832D091505040E695FF
:1020C000001CCAF72BD0FE2F29D0660F771F881F60
:1020D000BB1F261737074807AB07B0E809F0BB0B53
:1020E000802DBF01FF2793585F4F3AF09E3F510567
:1020F00078F00C9430110C947B115F3FE4F3983E20
:10210000D4F3869577956795B795F7959F5FC9F74F
:10211000880F911D9695879597F90895E1E0660FD0
:10212000771F881FBB1F621773078407BA0720F049
:10213000621B730B840BBA0BEE1F88F7E0950895B2
:102140000E94601188F09F5798F0B92F9927B751D6
:10215000B0F0E1F0660F771F881F991F1AF0BA954B
:10216000C9F714C0B13091F00E947A11B1E008951E
:102170000C947A11672F782F8827B85F39F0B93F10
:10218000CCF3869577956795B395D9F73EF49095FE
:102190008095709561957F4F8F4F9F4F0895E8947C
:1021A00009C097FB3EF490958095709561957F4F9F
:1021B0008F4F9F4F9923A9F0F92F96E9BB2793954D
:1021C000F695879577956795B795F111F8CFFAF45D
:1021D000BB0F11F460FF1BC06F5F7F4F8F4F9F4F8E
:1021E00016C0882311F096E911C0772321F09EE8EC
:1021F000872F762F05C0662371F096E8862F70E052
:1022000060E02AF09A95660F771F881FDAF7880F2B
:102210009695879597F90895990F0008550FAA0B81
:10222000E0E8FEEF16161706E807F907C0F01216E9
:102230001306E407F50798F0621B730B840B950BEC
:1022400039F40A2661F0232B242B252B21F4089541
:102250000A2609F4A140A6958FEF811D811D0895DE
:1022600097F99F6780E870E060E008959FEF80EC49
:10227000089500240A9416161706180609060895EC
:1022800000240A9412161306140605060895092E52
:102290000394000C11F4882352F0BB0F40F4BF2BC1
:1022A00011F460FF04C06F5F7F4F8F4F9F4F089501
:1022B00057FD9058440F551F59F05F3F71F04795F7
:1022C000880F97FB991F61F09F3F79F087950895DC
:1022D000121613061406551FF2CF4695F1DF08C0FB
:1022E000161617061806991FF1CF86957105610518
:1022F00008940895E894BB2766277727CB0197F9C0
:1023000008950E940C1108F48FEF089516F00C94B4
:1023100043120C94361168940C9430110E94601191
:10232000A8F39923C1F3AEF3DF93CF931F930F93D9
:10233000FF92C92FDD2788232AF02197660F771F88
:10234000881FDAF720E030E040E85FEB9FE3883950
:1023500020F0803E38F021968F770E94BD0FEEEB83
:10236000F0E004C00E94BD0FEBEEF0E00E945112BD
:102370008B01BE01EC01FB2E6F5771097595771F1C
:10238000880B990B0E94D11028E132E741E35FE30B
:102390000E94E911AF2D9801AE01FF900F911F919E
:1023A000CF91DF910E94D40F0C9447110E94E91144
:1023B0000C9447110E94391138F00E94401120F00E
:1023C000952311F00C9430110C94361111240C94B7
:1023D0007B110E94581170F3959FC1F3950F50E047
:1023E000551F629FF001729FBB27F00DB11D639FC7
:1023F000AA27F00DB11DAA1F649F6627B00DA11D6D
:10240000661F829F2227B00DA11D621F739FB00D12
:10241000A11D621F839FA00D611D221F749F332782
:10242000A00D611D231F849F600D211D822F762F1B
:102430006A2F11249F5750409AF0F1F088234AF0F8
:10244000EE0FFF1FBB1F661F771F881F9150504064
:10245000A9F79E3F510580F00C9430110C947B112C
:102460005F3FE4F3983ED4F3869577956795B795EB
:10247000F795E7959F5FC1F7FE2B880F911D969505
:10248000879597F908959F3F31F0915020F48795F3
:1024900077956795B795880F911D9695879597F9CC
:1024A0000895DF93CF931F930F93FF92EF92DF92E4
:1024B0007B018C01689406C0DA2EEF010E94E911BD
:1024C000FE01E894A5912591359145915591A6F38A
:1024D000EF010E94D40FFE019701A801DA9469F779
:1024E000DF90EF90FF900F911F91CF91DF910895B2
:1024F000EE0FFF1F0590F491E02D099481E090E02C
:0A250000F8940C948312F894FFCFB6
:10250A000101011E000C00E80300008041100000D8
:10251A00C040000000007B01E4001301C201440135
:04252A002201360153
:00000001FF
